:020000040000FA
:0408000054EF09F0B8
:1008100003B26DEF05F0F2B48BEF05F09EB093EFED
:1008200005F09EB29BEF05F0F2A81AEF04F0F2B2C9
:100830001CEF04F003EF09F0CD90F2929EA026EF9A
:1008400004F00101533F26EF04F0542BAEC1B2F186
:10085000AFC1B3F1B0C1B4F1B1C1B5F1AAC1AEF14C
:10086000ABC1AFF1ACC1B0F1ADC1B1F1A6C1AAF15C
:10087000A7C1ABF1A8C1ACF1A9C1ADF1A2C1A6F16C
:10088000A3C1A7F1A4C1A8F1A5C1A9F19EC1A2F17C
:100890009FC1A3F1A0C1A4F1A1C1A5F19AC19EF18C
:1008A0009BC19FF19CC1A0F19DC1A1F196C19AF19C
:1008B00097C19BF198C19CF199C19DF1CECF96F162
:1008C000CFCF97F153C198F154C199F1CF6ACE6A55
:1008D0000101536B546B9E90CD800FBC0F8E0FBAED
:1008E00075EF04F00F8A03EF09F00F8C0FBEB1EF24
:1008F00004F096C19AF197C19BF198C19CF199C1FE
:100900009DF19AC19EF19BC19FF19CC1A0F19DC137
:10091000A1F19EC1A2F19FC1A3F1A0C1A4F1A1C107
:10092000A5F1A2C1A6F1A3C1A7F1A4C1A8F1A5C1D7
:10093000A9F1A6C1AAF1A7C1ABF1A8C1ACF1A9C1A7
:10094000ADF1AAC1AEF1ABC1AFF1ACC1B0F1ADC177
:10095000B1F1AEC1B2F1AFC1B3F1B0C1B4F1B1C147
:10096000B5F101015E6B5F6B606B616B96515E2749
:1009700097515F2398516023995161239A515E27C3
:100980009B515F239C5160239D5161239E515E27A3
:100990009F515F23A0516023A1516123A2515E2783
:1009A000A3515F23A4516023A5516123A6515E2763
:1009B000A7515F23A8516023A9516123AA515E2743
:1009C000AB515F23AC516023AD516123AE515E2723
:1009D000AF515F23B0516023B1516123B2515E2703
:1009E000B3515F23B4516023B5516123D890010105
:1009F000613360335F335E33D8900101613360331C
:100A00005F335E33D8900101613360335F335E330F
:100A100000C10CF101C10DF102C10EF103C10FF1D2
:100A200004C110F105C111F106C112F107C113F1A2
:100A300008C114F109C115F10AC116F10BC117F172
:100A400034C135F111B830EF05F00101620E046FC9
:100A5000010E056F000E066F000E076F39EF05F0EF
:100A60000101A70E046F020E056F000E066F000E47
:100A7000076F5EC100F15FC101F160C102F161C1A8
:100A800003F131EC1FF003BF04D019BE02D019A04E
:100A9000108C11A051EF05F010BA51EF05F00F8046
:100AA000108A0CC100F10DC101F10EC102F10FC19C
:100AB00003F110C104F111C105F112C106F113C116
:100AC00007F114C108F115C109F116C10AF117C1E6
:100AD0000BF135C134F103EF09F00392ABB2AB98DF
:100AE000AB88030103EE00F080517F0BE92604C0C0
:100AF000EFFF802B8151805D700BD8A48B820000AA
:100B00008051815D700BD8A48B9281518019D8B42B
:100B1000079003EF09F0F2940101453F03EF09F05C
:100B2000462B03EF09F09E900101533F03EF09F0BC
:100B3000542B03EF09F09E9213A0C5EF05F00101BD
:100B40005E6B5F6B606B616B626B636B646B656B41
:100B5000666B676B686B696B536B546BCF6ACE6A5D
:100B60000F9A0F9C0F9E0101476B486B496B4A6BB4
:100B70004B6B4C6B4D6B4E6B4F6B506B516B526BA9
:100B8000456B466BD76AD66A139011B833EF07F0FE
:100B90008BB4D2EF05F010ACD2EF05F08B84109C33
:100BA000D3EF05F08B94C3CF55F1C4CF56F1C28279
:100BB00007B43DEF06F047C14BF148C14CF149C1C4
:100BC0004DF14AC14EF15EC162F15FC163F160C196
:100BD00064F161C165F196C1B6F197C1B7F198C1F1
:100BE000B8F199C1B9F19AC1BAF19BC1BBF19CC1ED
:100BF000BCF19DC1BDF19EC1BEF19FC1BFF1A0C1BD
:100C0000C0F1A1C1C1F1A2C1C2F1A3C1C3F1A4C18C
:100C1000C4F1A5C1C5F1A6C1C6F1A7C1C7F1A8C15C
:100C2000C8F1A9C1C9F1AAC1CAF1ABC1CBF1ACC12C
:100C3000CCF1ADC1CDF1AEC1CEF1AFC1CFF1B0C1FC
:100C4000D0F1B1C1D1F1B2C1D2F1B3C1D3F1B4C1CC
:100C5000D4F1B5C1D5F1010155515B2756515C2343
:100C6000E86A5D230E2E3DEF06F05CC157F15DC1D1
:100C700058F15B6B5C6B5D6B078E0201002F03EF1D
:100C800009F03C0E006F1A50E00BE00AE86612888B
:100C900018BE02D018B4108E00C10CF101C10DF1C4
:100CA00002C10EF103C10FF104C110F105C111F130
:100CB00006C112F107C113F108C114F109C115F100
:100CC0000AC116F10BC117F134C135F101018A6770
:100CD00071EF06F08B6771EF06F08C6771EF06F02D
:100CE0008D6775EF06F0A5EF06F08EC100F18FC19C
:100CF00001F190C102F191C103F10101010E046FF4
:100D0000000E056F000E066F000E076F31EC1FF02E
:100D100000C18EF101C18FF102C190F103C191F1C7
:100D200000679AEF06F001679AEF06F002679AEF04
:100D300006F00367A5EF06F08AC18EF18BC18FF133
:100D40008CC190F18DC191F10F80D57ED5BE6DD053
:100D5000D6CF47F1D7CF48F145C149F1E86AE8CF8E
:100D60004AF119BE02D019A0108C109047C100F1B1
:100D700048C101F149C102F14AC103F101010A0E62
:100D8000046F000E056F000E066F000E076F31EC4A
:100D90001FF003AF1080010154A7DBEF06F00F9A9C
:100DA0000F9C0F9E0101000E5E6F600E5F6F3D0E87
:100DB000606F080E616F010147BFEBEF06F04867F7
:100DC000EBEF06F04967EBEF06F04A67EBEF06F052
:100DD000F28810EF07F0F2985E6B5F6B606B616BEF
:100DE000966B976B986B996B9A6B9B6B9C6B9D6BDF
:100DF0009E6B9F6BA06BA16BA26BA36BA46BA56B8F
:100E0000A66BA76BA86BA96BAA6BAB6BAC6BAD6B3E
:100E1000AE6BAF6BB06BB16BB26BB36BB46BB56BEE
:100E2000D76AD66A0101456B466B0CC100F10DC152
:100E300001F10EC102F10FC103F110C104F111C1A2
:100E400005F112C106F113C107F114C108F115C172
:100E500009F116C10AF117C10BF135C134F103EFE5
:100E600009F003EF09F00201002F8CEF08F0D59E86
:100E7000D6CF47F1D7CF48F145C149F1E86AE8CF6D
:100E80004AF1D76AD66A0101456B466BD58E1A5076
:100E9000E00BE00AE866128818BE02D018B4108E83
:100EA00017AE1C8C00C10CF101C10DF102C10EF195
:100EB00003C10FF104C110F105C111F106C112F116
:100EC00007C113F108C114F109C115F10AC116F1E6
:100ED0000BC117F134C135F10FA0109A11B87CEF96
:100EE00007F00101620E046F010E056F000E066F20
:100EF000000E076F85EF07F00101A70E046F020EC9
:100F0000056F000E066F000E076F47C100F148C164
:100F100001F149C102F14AC103F131EC1FF003BFF5
:100F200098EF07F019BE02D019A0108C11B00F80F5
:100F30000CC100F10DC101F10EC102F10FC103F1AD
:100F400010C104F111C105F112C106F113C107F17D
:100F500014C108F115C109F116C10AF117C10BF14D
:100F600035C134F102013C0E006F00C10CF101C12A
:100F70000DF102C10EF103C10FF104C110F105C161
:100F800011F106C112F107C113F108C114F109C131
:100F900015F10AC116F10BC117F134C135F1010188
:100FA0008A67DAEF07F08B67DAEF07F08C67DAEF22
:100FB00007F08D67DEEF07F00EEF08F08EC100F14D
:100FC0008FC101F190C102F191C103F10101010E44
:100FD000046F000E056F000E066F000E076F31ECF8
:100FE0001FF000C18EF101C18FF102C190F103C168
:100FF00091F1006703EF08F0016703EF08F0026763
:1010000003EF08F003670EEF08F08AC18EF18BC181
:101010008FF18CC190F18DC191F10F80109047C17B
:1010200000F148C101F149C102F14AC103F10101D6
:101030000A0E046F000E056F000E066F000E076F9C
:1010400031EC1FF003AF1080010154A734EF08F01A
:101050000F9A0F9C0F9E0101000E5E6F600E5F6F76
:101060003D0E606F080E616F47C100F148C101F18C
:1010700049C102F14AC103F10101140E046F050ECA
:10108000056F000E066F000E076F31EC1FF003AF07
:101090004DEF08F0F28872EF08F0F2985E6B5F6B2C
:1010A000606B616B966B976B986B996B9A6B9B6B94
:1010B0009C6B9D6B9E6B9F6BA06BA16BA26BA36BDC
:1010C000A46BA56BA66BA76BA86BA96BAA6BAB6B8C
:1010D000AC6BAD6BAE6BAF6BB06BB16BB26BB36B3C
:1010E000B46BB56B0CC100F10DC101F10EC102F181
:1010F0000FC103F110C104F111C105F112C106F1D4
:1011000013C107F114C108F115C109F116C10AF1A3
:1011100017C10BF135C134F18BB496EF08F010AC68
:1011200096EF08F08B84109C97EF08F08B94C3CF58
:1011300055F1C4CF56F1C28207B401EF09F047C19F
:101140004BF148C14CF149C14DF14AC14EF15EC16C
:1011500062F15FC163F160C164F161C165F196C183
:10116000B6F197C1B7F198C1B8F199C1B9F19AC177
:10117000BAF19BC1BBF19CC1BCF19DC1BDF19EC147
:10118000BEF19FC1BFF1A0C1C0F1A1C1C1F1A2C117
:10119000C2F1A3C1C3F1A4C1C4F1A5C1C5F1A6C1E7
:1011A000C6F1A7C1C7F1A8C1C8F1A9C1C9F1AAC1B7
:1011B000CAF1ABC1CBF1ACC1CCF1ADC1CDF1AEC187
:1011C000CEF1AFC1CFF1B0C1D0F1B1C1D1F1B2C157
:1011D000D2F1B3C1D3F1B4C1D4F1B5C1D5F101019C
:1011E00055515B2756515C23E86A5D230E2E01EFB3
:1011F00009F05CC157F15DC158F15B6B5C6B5D6BD5
:10120000078E03EF09F002C0E0FF005001C0D8FFD5
:101210001000A6B209EF09F00CC0A9FF0BC0A8FF8F
:10122000A69EA69CA684F29E550EA76EAA0EA76E39
:10123000A682F28EA694A6B21BEF09F00C2A120029
:10124000A96EA69EA69CA680A8500C2A1200040196
:101250002C0E826F2FEC0BF02CEC20F00C5020ECBD
:1012600009F0E8CF00F10C5020EC09F0E8CF01F1D3
:1012700001AF40EF09F00101FF0E026FFF0E036F97
:10128000CFEC1FF029674CEF09F00401200E826FAC
:101290002FEC0BF051EF09F004012D0E826F2FECB3
:1012A0000BF0D9EC1DF01200306A076A0F6A106A61
:1012B000116A126A136A0F010E0EC16E860EC06E9D
:1012C000030EC26E0F01896A110E926E080E8A6EAD
:1012D000F10E936E8B6A800E946EF18E81848286FD
:1012E000FC0E20EC09F0E8CF0BF00BA011800BA254
:1012F00011820BA411840BA81188C90E20EC09F0EF
:10130000E8CF17F0CA0E20EC09F0E8CF18F0CB0EAA
:1013100020EC09F0E8CF19F0CC0E20EC09F0E8CF72
:101320001AF0CD0E20EC09F0E8CF2FF01C6A1D6AF0
:101330000E6A01015B6B5C6B5D6B576B586BF29ACD
:101340000101476B486B496B4A6B4B6B4C6B4D6BA8
:101350004E6B4F6B506B516B526B456B466BD76A44
:10136000D66A0F01280ED56EF28A9D90B00ECD6E12
:1013700001015E6B5F6B606B616B626B636B646BD7
:10138000656B666B676B686B696B536B546BCF6A8D
:10139000CE6A0F9A0F9C0F9E9D80760ECA6E9D821C
:1013A00002013C0E006FCC6A160E20EC09F0E8CF6B
:1013B00000F1170E20EC09F0E8CF01F1180E20EC37
:1013C00009F0E8CF02F1190E20EC09F0E8CF03F1A3
:1013D000010103AF06EF0AF02CEC20F0160E0C6EA4
:1013E00000C10BF009EC09F0170E0C6E01C10BF0F7
:1013F00009EC09F0180E0C6E02C10BF009EC09F0B3
:10140000190E0C6E03C10BF009EC09F000C18AF152
:1014100001C18BF102C18CF103C18DF100C18EF1CC
:1014200001C18FF102C190F103C191F11A0E20ECBC
:1014300009F0E8CF00F11B0E20EC09F0E8CF01F134
:101440001C0E20EC09F0E8CF02F11D0E20EC09F093
:10145000E8CF03F1010103AF5CEF0AF02CEC20F0C0
:101460001A0E0C6E00C10BF009EC09F01B0E0C6E8D
:1014700001C10BF009EC09F01C0E0C6E02C10BF05F
:1014800009EC09F01D0E0C6E03C10BF009EC09F01C
:101490001A0E20EC09F0E8CF00F11B0E20EC09F049
:1014A000E8CF01F11C0E20EC09F0E8CF02F11D0E8F
:1014B00020EC09F0E8CF03F100C192F101C193F1F2
:1014C00002C194F103C195F1240EAC6E900EAB6E87
:1014D000240EAC6E080EB86E000EB06E1F0EAF6E0E
:1014E0000401806B816B0F01900EAB6E0F019D8A22
:1014F0000301806B816BC26B8B9207900001F28EAF
:10150000F28C07B087EF1CF00FB01DEF16F010BE85
:101510001DEF16F012B81DEF16F00301805181196E
:101520007F0BD8B487EF1CF013EE00F081517F0BD6
:10153000E126812BE7CFE8FFE00BD8B487EF1CF062
:1015400023EE82F0C2513F0BD926E7CFDFFFC22B3B
:10155000DF50780AD8A487EF1CF007808EC100F115
:101560008FC101F190C102F191C103F10101040E9B
:10157000046F000E056F000E066F000E076F31EC52
:101580001FF000AFCDEF0AF00101030E8E6F000EC9
:101590008F6F000E906F000E916F03018251720ADF
:1015A000D8B402EF16F08251520AD8B402EF16F006
:1015B0008251750AD8B402EF16F08251630AD8B48A
:1015C00041EF19F08251690AD8B4B1EF12F082519B
:1015D0007A0AD8B4C4EF13F08251490AD8B402EFA2
:1015E00012F08251500AD8B420EF11F08251700AE3
:1015F000D8B463EF11F08251540AD8B48EEF11F0D1
:101600008251740AD8B4D4EF11F08251410AD8B48F
:1016100045EF0CF082514B0AD8B443EF0BF08251E6
:101620006D0AD8B478EF10F082514D0AD8B491EF1A
:1016300010F08251730AD8B432EF15F08251530A78
:10164000D8B497EF15F08251660AD8B463EF12F060
:101650008251590AD8B4C9EF0FF078EF19F004019C
:1016600014EE00F080517F0BE12682C4E7FF802B4F
:10167000120004010D0E826F2FEC0BF00A0E826F28
:101680002FEC0BF0120004014B0E826F2FEC0BF0CD
:1016900004012C0E826F2FEC0BF081B802D02FB614
:1016A00030D003018351430AD8B488EF0BF0030113
:1016B0008351630AD8B48AEF0BF003018351520AB5
:1016C000D8B48CEF0BF003018351720AD8B48EEFBB
:1016D0000BF003018351470AD8B490EF0BF00301DC
:1016E0008351670AD8B492EF0BF003018351540A77
:1016F000D8B494EF0BF003018351740AD8B403EF0C
:101700000CF003018351550AD8B496EF0BF082D048
:101710002F807AD02F9078D02F8276D02F9274D0CD
:101720002F8472D02F9470D02F866ED084C330F166
:1017300085C331F186C332F187C333F10101296BCF
:101740007AEC20F0F1EC1FF000C104F101C105F1C9
:1017500002C106F103C107F16DEC20F0200EF86E16
:10176000F76AF66A0900F5CF2CF10900F5CF2DF1E3
:101770000900F5CF2EF10900F5CF2FF10900F5CFC3
:1017800030F10900F5CF31F10900F5CF32F1090050
:10179000F5CF33F10101296B7AEC20F0F1EC1FF069
:1017A00031EC1FF00067DCEF0BF00167DCEF0BF0B2
:1017B0000267DCEF0BF0036701D025D004014E0E69
:1017C000826F2FEC0BF004016F0E826F2FEC0BF089
:1017D00004014D0E826F2FEC0BF00401610E826F3D
:1017E0002FEC0BF00401740E826F2FEC0BF0040150
:1017F000630E826F2FEC0BF00401680E826F2FECEA
:101800000BF076EF19F02F96CD0E0C6E2FC00BF06B
:1018100009EC09F0CD0E20EC09F0E8CF2FF02FB045
:1018200006D00401630E826F2FEC0BF005D004018B
:10183000430E826F2FEC0BF02FB206D00401720E14
:10184000826F2FEC0BF005D00401520E826F2FEC4B
:101850000BF02FB406D00401670E826F2FEC0BF053
:1018600005D00401470E826F2FEC0BF02FB606D087
:101870000401740E826F2FEC0BF005D00401540E9E
:10188000826F2FEC0BF076EF19F00401410E826F9E
:101890002FEC0BF003018351310AD8B4E9EF0EF0BD
:1018A00003018351320AD8B419EF0EF003018351BA
:1018B000330AD8B4A2EF0DF003018351340AD8B42F
:1018C00092EF0CF003018351350AD8B46FEF0CF09E
:1018D00004013F0E826F2FEC0BF076EF19F004013C
:1018E0002C0E826F2FEC0BF003018451300AD8B418
:1018F00082EF0CF003018451310AD8B48AEF0CF066
:10190000DBEF0DF08B900401300E826F2FEC0BF0AB
:1019100090EF0CF08B800401310E826F2FEC0BF0F6
:1019200076EF19F0CC0E20EC09F0E8CF0BF00401B3
:101930002C0E826F2FEC0BF003018451310AD8B4C6
:10194000B6EF0CF003018451300AD8B4B8EF0CF0B4
:10195000030184514D0AD8B4C2EF0CF00301845145
:10196000540AD8B4C9EF0CF0E0EF0CF08A8401D02F
:101970008A940BAE04D00BAC02D00BBA21D0E00E8F
:101980000B1218D01F0E0B168539E844E00B0B1212
:1019900011D0E00E0B166DEC20F085C332F186C33A
:1019A00033F10101296B7AEC20F0F1EC1FF00051CA
:1019B0001F0B0B12CC0E0C6E0BC00BF009EC09F0D8
:1019C0000401340E826F2FEC0BF004012C0E826F99
:1019D0002FEC0BF0CC0E20EC09F0E8CF1AF08AB413
:1019E00006D00401300E826F2FEC0BF005D00401FD
:1019F000310E826F2FEC0BF004012C0E826F2FEC56
:101A00000BF01A38E840070BE8CF82F40401300EDF
:101A100082272FEC0BF004012C0E826F2FEC0BF0C1
:101A20002CEC20F01A501F0BE8CF00F1CFEC1FF088
:101A300032C182F40401300E82272FEC0BF033C147
:101A400082F40401300E82272FEC0BF004012C0EDF
:101A5000826F2FEC0BF02CEC20F02DC000F100AFCA
:101A60000BD0FF0E016FFF0E026FFF0E036F04011C
:101A70002D0E826F2FEC0BF0CFEC1FF031C182F4F2
:101A80000401300E82272FEC0BF032C182F40401E6
:101A9000300E82272FEC0BF033C182F40401300E9C
:101AA00082272FEC0BF004012C0E826F2FEC0BF031
:101AB0002CEC20F02CC000F1CFEC1FF031C182F4EF
:101AC0000401300E82272FEC0BF032C182F40401A6
:101AD000300E82272FEC0BF033C182F40401300E5C
:101AE00082272FEC0BF004012C0E826F2FEC0BF0F1
:101AF0002CEC20F02EC000F100AF0BD0FF0E016FD8
:101B0000FF0E026FFF0E036F04012D0E826F2FEC8C
:101B10000BF0CFEC1FF031C182F40401300E8227AC
:101B20002FEC0BF032C182F40401300E82272FEC2F
:101B30000BF033C182F40401300E82272FEC0BF03E
:101B400076EF19F0CB0E20EC09F0E8CF0BF0040192
:101B50002C0E826F2FEC0BF003018451450AD8B490
:101B6000C6EF0DF003018451440AD8B4C9EF0DF05B
:101B700003018451300AD8B4CCEF0DF00301845135
:101B8000310AD8B4D0EF0DF0DBEF0DF00B9ED5EF9E
:101B90000DF00B8ED5EF0DF0FC0E0B16D5EF0DF002
:101BA000FC0E0B160B80D5EF0DF0CB0E0C6E0BC0A0
:101BB0000BF009EC09F00401330E826F2FEC0BF0EF
:101BC00004012C0E826F2FEC0BF0CB0E20EC09F0F1
:101BD000E8CF19F019BEF4EF0DF00401450E826F45
:101BE0002FEC0BF0F9EF0DF00401440E826F2FEC97
:101BF0000BF004012C0E826F2FEC0BF00401300E61
:101C0000826F2FEC0BF004012C0E826F2FEC0BF087
:101C100019B012EF0EF00401300E826F2FEC0BF0B2
:101C200017EF0EF00401310E826F2FEC0BF076EF00
:101C300019F0CA0E20EC09F0E8CF0BF004012C0ECD
:101C4000826F2FEC0BF003018451450AD8B455EF95
:101C50000EF003018451440AD8B458EF0EF003018A
:101C600084514D0AD8B461EF0EF003018451410A4A
:101C7000D8B45BEF0EF003018451460AD8B45EEF8E
:101C80000EF003018451560AD8B469EF0EF0030137
:101C90008451500AD8B474EF0EF003018451520AF3
:101CA000D8B477EF0EF080EF0EF00B9E7AEF0EF0C7
:101CB0000B8E7AEF0EF00B9C7AEF0EF00B8C7AEF16
:101CC0000EF0FC0E0B1685C3E8FF030B0B127AEF28
:101CD0000EF0C70E0B1685C3E8FF070BE846E84673
:101CE000E8460B127AEF0EF00B847AEF0EF00B94AD
:101CF0007AEF0EF0CA0E0C6E0BC00BF009EC09F077
:101D0000CA0E20EC09F0E8CF18F00401320E826F01
:101D10002FEC0BF004012C0E826F2FEC0BF018BE91
:101D200099EF0EF00401450E826F2FEC0BF09EEF41
:101D30000EF00401440E826F2FEC0BF004012C0E08
:101D4000826F2FEC0BF018C0E8FF030BE8CF82F492
:101D50000401300E82272FEC0BF004012C0E826F51
:101D60002FEC0BF018BCBCEF0EF00401410E826F9B
:101D70002FEC0BF0C1EF0EF00401460E826F2FEC3A
:101D80000BF004012C0E826F2FEC0BF018C0E8FF53
:101D9000380BE842E842E842E8CF82F40401300E12
:101DA00082272FEC0BF004012C0E826F2FEC0BF02E
:101DB00018B4E2EF0EF00401520E826F2FEC0BF01C
:101DC000E7EF0EF00401500E826F2FEC0BF076EF70
:101DD00019F0C90E20EC09F0E8CF0BF004012C0E2D
:101DE000826F2FEC0BF003018451450AD8B407EF42
:101DF0000FF003018451440AD8B40AEF0FF0030135
:101E000084514D0AD8B40DEF0FF01BEF0FF00B9E6D
:101E100015EF0FF00B8E15EF0FF0F80E0B1685C3B4
:101E2000E8FF070B0B1215EF0FF0C90E0C6E0BC07D
:101E30000BF009EC09F00401310E826F2FEC0BF06E
:101E400004012C0E826F2FEC0BF0C90E20EC09F070
:101E5000E8CF17F017BE06D00401450E826F2FECB5
:101E60000BF005D00401440E826F2FEC0BF004013F
:101E70002C0E826F2FEC0BF017C0E8FF070BE8CF9A
:101E800082F40401300E82272FEC0BF004012C0E9B
:101E9000826F2FEC0BF007802CEC20F028C0E8FFBD
:101EA000003B00430043030BCFEC1FF033C182F42F
:101EB0000401300E82272FEC0BF004012C0E826FF0
:101EC0002FEC0BF02CEC20F028C001F1019F019DBC
:101ED00029C000F10101CFEC1FF02FC182F40401F1
:101EE000300E82272FEC0BF030C182F40401300E4B
:101EF00082272FEC0BF031C182F40401300E8227CF
:101F00002FEC0BF032C182F40401300E82272FEC4B
:101F10000BF033C182F40401300E82272FEC0BF05A
:101F200004012C0E826F2FEC0BF02CEC20F02AC059
:101F300001F12BC000F1D89001330033D890013368
:101F400000330101CFEC1FF02FC182F40401300EE9
:101F500082272FEC0BF030C182F40401300E82276F
:101F60002FEC0BF031C182F40401300E82272FECEC
:101F70000BF032C182F40401300E82272FEC0BF0FB
:101F800033C182F40401300E82272FEC0BF076EF80
:101F900019F0FC0E20EC09F0E8CF0BF0030183519F
:101FA000520AD8B400EF10F003018351720AD8B47A
:101FB00003EF10F003018351500AD8B406EF10F07C
:101FC00003018351700AD8B409EF10F00301835163
:101FD000550AD8B40CEF10F003018351750AD8B438
:101FE0000FEF10F003018351430AD8B418EF10F03B
:101FF00003018351630AD8B41BEF10F024EF10F0F3
:102000000B901EEF10F00B801EEF10F00B921EEFE6
:1020100010F00B821EEF10F00B941EEF10F00B84EB
:102020001EEF10F00B961EEF10F00B861EEF10F057
:102030000B981EEF10F00B881EEF10F0FC0E0C6ECC
:102040000BC00BF009EC09F00401590E826F2FEC64
:102050000BF01190119211941198FC0E20EC09F0E4
:10206000E8CF0BF00BA011800BA211820BA41184FE
:102070000BA8118811A044EF10F00401520E826FDA
:102080002FEC0BF049EF10F00401720E826F2FEC71
:102090000BF011A853EF10F00401430E826F2FECE8
:1020A0000BF058EF10F00401630E826F2FEC0BF071
:1020B00011A262EF10F00401500E826F2FEC0BF0B2
:1020C00067EF10F00401700E826F2FEC0BF011A47B
:1020D00071EF10F00401550E826F2FEC0BF076EFCC
:1020E00010F00401750E826F2FEC0BF076EF19F0F3
:1020F00004016D0E826F2FEC0BF003018351300A47
:10210000D8B4D0EF10F003018351310AD8B4E3EF13
:1021100010F003018351320AD8B4F6EF10F078EFD3
:1021200019F004014D0E826F2FEC0BF06DEC20F0D6
:1021300084C331F185C332F186C333F10101296BC8
:102140007AEC20F0F1EC1FF003018351300AD8B48F
:10215000B8EF10F003018351310AD8B4C0EF10F08A
:1021600003018351320AD8B4C8EF10F078EF19F0A8
:10217000FD0E0C6E00C10BF009EC09F0D0EF10F071
:10218000FE0E0C6E00C10BF009EC09F0E3EF10F04D
:10219000FF0E0C6E00C10BF009EC09F0F6EF10F029
:1021A0000401300E826F2FEC0BF004012C0E826FB5
:1021B0002FEC0BF02CEC20F0FD0E20EC09F0E8CF1A
:1021C00000F107EF11F00401310E826F2FEC0BF0DC
:1021D00004012C0E826F2FEC0BF02CEC20F0FE0E85
:1021E00020EC09F0E8CF00F107EF11F00401320E06
:1021F000826F2FEC0BF02CEC20F004012C0E826F80
:102200002FEC0BF0FF0E20EC09F0E8CF00F1CFEC43
:102210001FF031C182F40401300E82272FEC0BF045
:1022200032C182F40401300E82272FEC0BF033C14F
:1022300082F40401300E82272FEC0BF076EF19F0B8
:1022400083C32AF184C32BF185C32CF186C32DF1FE
:1022500087C32EF188C32FF189C330F18AC331F1CE
:102260008BC332F18CC333F101017AEC20F0F1EC35
:102270001FF0160E0C6E00C10BF009EC09F0170EE2
:102280000C6E01C10BF009EC09F0180E0C6E02C1C6
:102290000BF009EC09F0190E0C6E03C10BF009EC00
:1022A00009F000C18AF101C18BF102C18CF103C1B7
:1022B0008DF100C18EF101C18FF102C190F103C116
:1022C00091F102EF12F083C32AF184C32BF185C38D
:1022D0002CF186C32DF187C32EF188C32FF189C35A
:1022E00030F18AC331F18BC332F18CC333F1010178
:1022F0007AEC20F0F1EC1FF000C18AF101C18BF102
:1023000002C18CF103C18DF100C18EF101C18FF1C9
:1023100002C190F103C191F102EF12F083C32AF1DF
:1023200084C32BF185C32CF186C32DF187C32EF115
:1023300088C32FF189C330F18AC331F18CC332F1E4
:102340008DC333F101017AEC20F0F1EC1FF00101B3
:10235000000E046F000E056F010E066F000E076F72
:1023600042EC1FF01A0E0C6E00C10BF009EC09F0E4
:102370001B0E0C6E01C10BF009EC09F01C0E0C6E6B
:1023800002C10BF009EC09F01D0E0C6E03C10BF03D
:1023900009EC09F000C192F101C193F102C194F17D
:1023A00003C195F102EF12F083C32AF184C32BF12C
:1023B00085C32CF186C32DF187C32EF188C32FF17D
:1023C00089C330F18AC331F18CC332F18DC333F14B
:1023D00001017AEC20F0F1EC1FF00101000E046F16
:1023E000000E056F010E066F000E076F42EC1FF026
:1023F00000C192F101C193F102C194F103C195F1C1
:1024000002EF12F0160E20EC09F0E8CF00F1170EE3
:1024100020EC09F0E8CF01F1180E20EC09F0E8CF2C
:1024200002F1190E20EC09F0E8CF03F1CFEC1FF018
:1024300092EC1DF00401730E826F2FEC0BF004017F
:102440002C0E826F2FEC0BF08AC100F18BC101F1D1
:102450008CC102F18DC103F1CFEC1FF092EC1DF0A5
:102460000401730E826F2FEC0BF004012C0E826FAF
:102470002FEC0BF01A0E20EC09F0E8CF00F11B0E48
:1024800020EC09F0E8CF01F11C0E20EC09F0E8CFB8
:1024900002F11D0E20EC09F0E8CF03F193EC19F0E6
:1024A00004012C0E826F2FEC0BF092C100F193C14E
:1024B00001F194C102F195C103F193EC19F039ECEB
:1024C0000BF078EF19F00401660E826F2FEC0BF021
:1024D00003018351780AD8B484EF12F0030183B169
:1024E00002D0829601D0828683B302D0819401D03B
:1024F000818484B102D0829A01D0828A84B302D0CE
:10250000829801D08288138088EC12F076EF19F05F
:1025100004012C0E826F2FEC0BF0300E82B602D02D
:10252000E89001D0E88081B402D0E89201D0E8823E
:10253000E8CF82F42FEC0BF004012C0E826F2FEC0D
:102540000BF0300E82BA02D0E89001D0E88082B859
:1025500002D0E89201D0E882E8CF82F42FEC0BF0B1
:1025600012000401690E826F2FEC0BF004012C0E97
:10257000826F2FEC0BF00101040E006F000E016F53
:10258000000E026F000E036FCFEC1FF02CC182F41F
:102590000401300E82272FEC0BF02DC182F40401D0
:1025A000300E82272FEC0BF02EC182F40401300E86
:1025B00082272FEC0BF02FC182F40401300E82270A
:1025C0002FEC0BF030C182F40401300E82272FEC87
:1025D0000BF031C182F40401300E82272FEC0BF096
:1025E00032C182F40401300E82272FEC0BF033C18C
:1025F00082F40401300E82272FEC0BF004012C0E24
:10260000826F2FEC0BF00101040E006F000E016FC2
:10261000000E026F000E036FCFEC1FF02CC182F48E
:102620000401300E82272FEC0BF02DC182F404013F
:10263000300E82272FEC0BF02EC182F40401300EF5
:1026400082272FEC0BF02FC182F40401300E822779
:102650002FEC0BF030C182F40401300E82272FECF6
:102660000BF031C182F40401300E82272FEC0BF005
:1026700032C182F40401300E82272FEC0BF033C1FB
:1026800082F40401300E82272FEC0BF004012C0E93
:10269000826F2FEC0BF00101360E006F000E016F00
:1026A000000E026F000E036FCFEC1FF02CC182F4FE
:1026B0000401300E82272FEC0BF02DC182F40401AF
:1026C000300E82272FEC0BF02EC182F40401300E65
:1026D00082272FEC0BF02FC182F40401300E8227E9
:1026E0002FEC0BF030C182F40401300E82272FEC66
:1026F0000BF031C182F40401300E82272FEC0BF075
:1027000032C182F40401300E82272FEC0BF033C16A
:1027100082F40401300E82272FEC0BF004012C0E02
:10272000826F2FEC0BF0200EF86EF76AF66A040148
:102730000900F5CF82F42FEC0BF00900F5CF82F4FD
:102740002FEC0BF00900F5CF82F42FEC0BF0090011
:10275000F5CF82F42FEC0BF00900F5CF82F42FECCB
:102760000BF00900F5CF82F42FEC0BF00900F5CF48
:1027700082F42FEC0BF00900F5CF82F42FEC0BF074
:1027800039EC0BF078EF19F08351630AD8A476EF97
:1027900019F08451610AD8A476EF19F085516C0ABA
:1027A000D8A476EF19F08651410A3FE08651440AD9
:1027B0001BE08651420AD8B428EF14F08651350A3E
:1027C000D8B402EF1BF08651360AD8B457EF1BF08D
:1027D0008651370AD8B4C0EF1BF08651380AD8B4F6
:1027E0001EEF1CF076EF19F00798079A04017A0E95
:1027F000826F2FEC0BF00401780E826F2FEC0BF040
:102800000401640E826F2FEC0BF00401550E826FF1
:102810002FEC0BF011EF14F004014C0E826F2FEC33
:102820000BF039EC0BF078EF19F00788079A0401E8
:102830007A0E826F2FEC0BF00401410E826F2FECA9
:102840000BF00401610E826F2FEC0BF005EF14F01A
:102850000798078A04017A0E826F2FEC0BF00401AF
:10286000420E826F2FEC0BF00401610E826F2FEC91
:102870000BF005EF14F00101666746EF14F067678F
:1028800046EF14F0686746EF14F0696715D04F679C
:1028900051EF14F0506751EF14F0516751EF14F0FD
:1028A00052670AD00101000E006F000E016F000E8A
:1028B000026F000E036F120011B80AD00101620E00
:1028C000046F010E056F000E066F000E076F09D032
:1028D0000101A70E046F020E056F000E066F000EB9
:1028E000076F66C100F167C101F168C102F169C1FA
:1028F00003F131EC1FF003BFEEEF14F0119A119CBD
:102900000101000E046FA80E056F550E066F020E32
:10291000076F66C100F167C101F168C102F169C1C9
:1029200003F166C186F167C187F168C188F169C1A9
:1029300089F131EC1FF003BF0BD00101000E866F4F
:10294000A80E876F550E886F020E896F118A119C31
:102950000E0E20EC09F0E8CF18F10F0E20EC09F074
:10296000E8CF19F1100E20EC09F0E8CF1AF1110EA2
:1029700020EC09F0E8CF1BF17AEC1EF086C104F1DF
:1029800087C105F188C106F189C107F131EC1FF05B
:1029900007823EEC1EF07AEC1EF007923EEC1EF031
:1029A00086C100F187C101F188C102F189C103F13B
:1029B00007923EEC1EF0CC0E046FE00E056F870E02
:1029C000066F050E076F31EC1FF000C118F101C151
:1029D00019F102C11AF103C11BF13BD0119C119AEC
:1029E0000101800E006F1A0E016F060E026F000EBD
:1029F000036F4FC104F150C105F151C106F152C13D
:102A000007F131EC1FF003AF05D02CEC20F0118C56
:102A1000119A12000E0E20EC09F0E8CF18F10F0EFB
:102A200020EC09F0E8CF19F1100E20EC09F0E8CF06
:102A30001AF1110E20EC09F0E8CF1BF14FC100F1A3
:102A400050C101F151C102F152C103F107823EECC4
:102A50001EF018C100F119C101F11AC102F11BC128
:102A600003F112000401730E826F2FEC0BF00401CE
:102A70002C0E826F2FEC0BF0078462C166F163C1EC
:102A800067F164C168F165C169F14BC14FF14CC197
:102A900050F14DC151F14EC152F157C159F158C1D8
:102AA0005AF1079458EC15F039EC0BF078EF19F067
:102AB00066C100F167C101F168C102F169C103F1AA
:102AC0000101CFEC1FF092EC1DF00401630E826F48
:102AD0002FEC0BF004012C0E826F2FEC0BF04FC18A
:102AE00000F150C101F151C102F152C103F10101E4
:102AF000CFEC1FF092EC1DF00401660E826F2FECFC
:102B00000BF004012C0E826F2FEC0BF02CEC20F05C
:102B100059C100F15AC101F10101CFEC1FF092EC53
:102B20001DF00401740E826F2FEC0BF01200108266
:102B30000401530E826F2FEC0BF004012C0E826FF8
:102B40002FEC0BF083C32AF184C32BF185C32CF146
:102B500086C32DF187C32EF188C32FF189C330F1CD
:102B60008AC331F18BC332F18CC333F101017AECAA
:102B700020F0F1EC1FF000C166F101C167F102C164
:102B800068F103C169F18EC32AF18FC32BF190C3A1
:102B90002CF191C32DF192C32EF193C32FF194C365
:102BA00030F195C331F196C332F197C333F101018E
:102BB0007AEC20F0F1EC1FF000C14FF101C150F1AF
:102BC00002C151F103C152F16DEC20F099C32FF114
:102BD0009AC330F19BC331F19CC332F19DC333F1F1
:102BE00001017AEC20F0F1EC1FF000C159F101C1B4
:102BF0005AF158EC15F004012C0E826F2FEC0BF0FB
:102C000011EF16F0118E19A002D019AE108C18BE5B
:102C100002D018A4108E8251520A02E10F8201D014
:102C20000F928251750A02E1108401D010948251F2
:102C3000550A02E1108601D0109611A003D011A40C
:102C400001D01084078410B27FEF16F010A46BEF50
:102C500016F0B6C166F1B7C167F1B8C168F1B9C184
:102C600069F1BAC16AF1BBC16BF1BCC16CF1BDC104
:102C70006DF1BEC16EF1BFC16FF1C0C170F1C1C1D4
:102C800071F1C2C172F1C3C173F1C4C174F1C5C1A4
:102C900075F1C6C176F1C7C177F1C8C178F1C9C174
:102CA00079F1CAC17AF1CBC17BF1CCC17CF1CDC144
:102CB0007DF1CEC17EF1CFC17FF1D0C180F1D1C114
:102CC00081F1D2C182F1D3C183F1D4C184F1D5C1E4
:102CD00085F173EF16F062C166F163C167F164C1FB
:102CE00068F165C169F14BC14FF14CC150F14DC163
:102CF00051F14EC152F157C159F158C15AF10794DF
:102D00000FA0A1EF16F0010192678EEF16F0936706
:102D10008EEF16F094678EEF16F0956792EF16F02F
:102D2000A1EF16F03BEC14F092C104F193C105F150
:102D300094C106F195C107F131EC1FF003BF3EEFDE
:102D400019F03BEC14F00101000E046F000E056F4A
:102D5000010E066F000E076F62EC1FF011A02AD063
:102D600011A228D0CFEC1FF0296701D005D00401B3
:102D70002D0E826F2FEC0BF030C182F40401300E67
:102D800082272FEC0BF031C182F40401300E822730
:102D90002FEC0BF032C182F40401300E82272FECAD
:102DA0000BF033C182F40401300E82272FEC0BF0BC
:102DB00039EC0BF012A8C3D012981AC01BF01B3AC2
:102DC0001B42070E1B1600011B50000AD8B46DEF02
:102DD00017F000011B50010AD8B4F9EF16F00001FA
:102DE0001B50020AD8B4F7EF16F09FEF17F09FEFD1
:102DF00017F02CEC20F02AC001F12BC000F1D89084
:102E000001330033D890013300330101630E046FA6
:102E1000000E056F000E066F000E076F62EC1FF0CC
:102E2000280E046F000E056F000E066F000E076F70
:102E300031EC1FF000C12DF02CEC20F028C001F186
:102E4000019F019D29C000F10101A40E046F000E35
:102E5000056F000E066F000E076F62EC1FF000C1D9
:102E60002CF000C104F101C105F102C106F103C15A
:102E700007F1640E006F000E016F000E026F000E6E
:102E8000036F31EC1FF0050E046F000E056F000E8E
:102E9000066F000E076F62EC1FF000C104F101C164
:102EA00005F102C106F103C107F12CEC20F02DC0A1
:102EB00000F131EC1FF000C12EF02EC0E8FF050F2D
:102EC0002D5C03E78A849FEF17F02EC0E8FF0A0FFE
:102ED0002D5C01E68A949FEF17F000C124F101C137
:102EE00025F102C126F103C127F12CEC20F032ECD0
:102EF00020F01A501F0BE8CF00F10101640E046F9F
:102F0000000E056F000E066F000E076F42EC1FF0FB
:102F100024C104F125C105F126C106F127C107F13D
:102F200031EC1FF003BF02D08A9401D08A8424C1FF
:102F300000F125C101F126C102F127C103F100C151
:102F400024F101C125F102C126F103C127F110AE20
:102F50004DD0109E00C108F101C109F102C10AF172
:102F600003C10BF1CFEC1FF030C1D6F131C1D7F165
:102F700032C1D8F133C1D9F108C100F109C101F161
:102F80000AC102F10BC103F101016C0E046F070EBF
:102F9000056F000E066F000E076F31EC1FF003BFC8
:102FA00004D00101550EDA6F1CD008C100F109C12F
:102FB00001F10AC102F10BC103F10101A40E046F7A
:102FC000060E056F000E066F000E076F31EC1FF046
:102FD00003BF04D001017F0EDA6F03D00101FF0EA1
:102FE000DA6F1C8E11AE3EEF19F0119E24C100F174
:102FF00025C101F126C102F127C103F111A005D0BD
:1030000011A203D00FB03EEF19F010A40FEF18F08B
:103010000401750E826F2FEC0BF014EF18F0040111
:10302000720E826F2FEC0BF004012C0E826F2FECCE
:103030000BF0CFEC1FF0296723EF18F00401200EEE
:10304000826F26EF18F004012D0E826F2FEC0BF02B
:1030500030C182F40401300E82272FEC0BF031C115
:1030600082F40401300E82272FEC0BF004012E0EA7
:10307000826F2FEC0BF032C182F40401300E8227F4
:103080002FEC0BF033C182F40401300E82272FECB9
:103090000BF004016D0E826F2FEC0BF004012C0E6F
:1030A000826F2FEC0BF04FC100F150C101F151C103
:1030B00002F152C103F10101CFEC1FF092EC1DF0BF
:1030C0000401480E826F2FEC0BF004017A0E826F20
:1030D0002FEC0BF004012C0E826F2FEC0BF066C16D
:1030E00000F167C101F168C102F169C103F1010199
:1030F000CFEC1FF092EC1DF00401630E826F2FECF9
:103100000BF004012C0E826F2FEC0BF066C100F166
:1031100067C101F168C102F169C103F101010A0E41
:10312000046F000E056F000E066F000E076F42EC75
:103130001FF0000E046F120E056F000E066F000EDA
:10314000076F62EC1FF0CFEC1FF02AC182F404017C
:10315000300E82272FEC0BF02BC182F40401300ECD
:1031600082272FEC0BF02CC182F40401300E822751
:103170002FEC0BF02DC182F40401300E82272FECCE
:103180000BF02EC182F40401300E82272FEC0BF0DD
:103190002FC182F40401300E82272FEC0BF030C1D6
:1031A00082F40401300E82272FEC0BF004012E0E66
:1031B000826F2FEC0BF031C182F40401300E8227B4
:1031C0002FEC0BF032C182F40401300E82272FEC79
:1031D0000BF033C182F40401300E82272FEC0BF088
:1031E0000401730E826F2FEC0BF004012C0E826F22
:1031F0002FEC0BF02CEC20F059C100F15AC101F179
:10320000A2EC1AF088EC12F00FB20AEF19F00FA03E
:103210003CEF19F004012C0E826F2FEC0BF0200E06
:10322000F86EF76AF66A04010900F5CF82F42FEC14
:103230000BF00900F5CF82F42FEC0BF00900F5CF6D
:1032400082F42FEC0BF00900F5CF82F42FEC0BF099
:103250000900F5CF82F42FEC0BF00900F5CF82F4D2
:103260002FEC0BF00900F5CF82F42FEC0BF00900E6
:10327000F5CF82F42FEC0BF039EC0BF00F9078EFD8
:1032800019F00401630E826F2FEC0BF004012C0E79
:10329000826F2FEC0BF07EEC19F004012C0E826F84
:1032A0002FEC0BF0F1EC19F004012C0E826F2FECD7
:1032B0000BF06DEC1AF004012C0E826F2FEC0BF06A
:1032C0000101F80E006FCD0E016F660E026F030E46
:1032D000036F93EC19F004012C0E826F2FEC0BF0AE
:1032E00083EC1AF039EC0BF078EF19F039EC0BF0B5
:1032F0000301C26B0790109287EF1CF0D8900E0E5E
:1033000020EC09F0E8CF00F10F0E20EC09F0E8CF37
:1033100001F1100E20EC09F0E8CF02F1110E20ECC3
:1033200009F0E8CF03F10101000E046F000E056FF4
:10333000010E066F000E076F62EC1FF0CFEC1FF05E
:103340002AC182F40401300E82272FEC0BF02BC12E
:1033500082F40401300E82272FEC0BF02CC182F492
:103360000401300E82272FEC0BF02DC182F40401F2
:10337000300E82272FEC0BF02EC182F40401300EA8
:1033800082272FEC0BF02FC182F40401300E82272C
:103390002FEC0BF030C182F40401300E82272FECA9
:1033A0000BF031C182F40401300E82272FEC0BF0B8
:1033B00004012E0E826F2FEC0BF032C182F4040157
:1033C000300E82272FEC0BF033C182F40401300E53
:1033D00082272FEC0BF004016D0E826F2FEC0BF0A7
:1033E0001200120E20EC09F0E8CF00F1130E20ECD1
:1033F00009F0E8CF01F1140E20EC09F0E8CF02F15A
:10340000150E20EC09F0E8CF03F101010A0E046F5C
:10341000000E056F000E066F000E076F42EC1FF0E6
:10342000000E046F120E056F000E066F000E076F80
:1034300062EC1FF0CFEC1FF02AC182F40401300EC1
:1034400082272FEC0BF02BC182F40401300E82276F
:103450002FEC0BF02CC182F40401300E82272FECEC
:103460000BF02DC182F40401300E82272FEC0BF0FB
:103470002EC182F40401300E82272FEC0BF02FC1F5
:1034800082F40401300E82272FEC0BF030C182F45D
:103490000401300E82272FEC0BF004012E0E826FF8
:1034A0002FEC0BF031C182F40401300E82272FEC97
:1034B0000BF032C182F40401300E82272FEC0BF0A6
:1034C00033C182F40401300E82272FEC0BF004018B
:1034D000730E826F2FEC0BF012000A0E20EC09F035
:1034E000E8CF00F10B0E20EC09F0E8CF01F10C0E53
:1034F00020EC09F0E8CF02F10D0E20EC09F0E8CF46
:1035000003F1A2EF1AF0060E20EC09F0E8CF00F16B
:10351000070E20EC09F0E8CF01F1080E20EC09F0CD
:10352000E8CF02F1090E20EC09F0E8CF03F1A2EF99
:103530001AF001012CEC20F0078457C100F158C1AA
:1035400001F107940101E80E046F800E056F000E73
:10355000066F000E076F42EC1FF0000E046F040EA2
:10356000056F000E066F000E076F62EC1FF0880EED
:10357000046F130E056F000E066F000E076F31EC1F
:103580001FF00A0E046F000E056F000E066F000E8E
:10359000076F62EC1FF0CFEC1FF001012967D6EF37
:1035A0001AF00401200E826FD9EF1AF004012D0EDB
:1035B000826F2FEC0BF030C182F40401300E8227B1
:1035C0002FEC0BF031C182F40401300E82272FEC76
:1035D0000BF032C182F40401300E82272FEC0BF085
:1035E00004012E0E826F2FEC0BF033C182F4040124
:1035F000300E82272FEC0BF00401430E826F2FEC6C
:103600000BF0120087C32AF188C32BF189C32CF178
:103610008AC32DF18BC32EF18CC32FF18DC330F1F2
:103620008EC331F190C332F191C333F10101296BA3
:103630007AEC20F0F1EC1FF00101000E046F000E97
:10364000056F010E066F000E076F42EC1FF00E0EA5
:103650000C6E00C10BF009EC09F00F0E0C6E01C1ED
:103660000BF009EC09F0100E0C6E02C10BF009EC26
:1036700009F0110E0C6E03C10BF009EC09F0040106
:103680007A0E826F2FEC0BF004012C0E826F2FEC60
:103690000BF00401350E826F2FEC0BF004012C0EA1
:1036A000826F2FEC0BF07EEC19F011EF14F087C352
:1036B0002AF188C32BF189C32CF18AC32DF18BC366
:1036C0002EF18CC32FF18DC330F18EC331F190C335
:1036D00032F191C333F10101296B7AEC20F0F1EC66
:1036E0001FF0880E046F130E056F000E066F000E9C
:1036F000076F36EC1FF0000E046F040E056F000E0E
:10370000066F000E076F42EC1FF00101E80E046F18
:10371000800E056F000E066F000E076F62EC1FF043
:103720000A0E0C6E00C10BF009EC09F00B0E0C6ECA
:1037300001C10BF009EC09F00C0E0C6E02C10BF08C
:1037400009EC09F00D0E0C6E03C10BF009EC09F049
:1037500004017A0E826F2FEC0BF004012C0E826FA5
:103760002FEC0BF00401360E826F2FEC0BF00401EE
:103770002C0E826F2FEC0BF06DEC1AF011EF14F0A1
:1037800087C32AF188C32BF189C32CF18AC32DF199
:103790008BC32EF18CC32FF18DC330F18FC331F168
:1037A00090C332F191C333F101017AEC20F0F1ECD6
:1037B0001FF0000E046F120E056F000E066F000E54
:1037C000076F42EC1FF001010A0E046F000E056F37
:1037D000000E066F000E076F62EC1FF0120E0C6EEB
:1037E00000C10BF009EC09F0130E0C6E01C10BF0D7
:1037F00009EC09F0140E0C6E02C10BF009EC09F093
:10380000150E0C6E03C10BF009EC09F004017A0EE1
:10381000826F2FEC0BF004012C0E826F2FEC0BF05B
:103820000401370E826F2FEC0BF004012C0E826F17
:103830002FEC0BF0F1EC19F011EF14F087C32AF123
:1038400088C32BF189C32CF18AC32DF18BC32EF1D0
:103850008CC32FF18DC330F18EC331F190C332F19F
:1038600091C333F10101296B7AEC20F0F1EC1FF0E8
:10387000880E046F130E056F000E066F000E076FA3
:1038800036EC1FF0000E046F040E056F000E066F7D
:10389000000E076F42EC1FF00101E80E046F800E6E
:1038A000056F000E066F000E076F62EC1FF0060E2C
:1038B0000C6E00C10BF009EC09F0070E0C6E01C193
:1038C0000BF009EC09F0080E0C6E02C10BF009ECCC
:1038D00009F0090E0C6E03C10BF009EC09F00401AC
:1038E0007A0E826F2FEC0BF004012C0E826F2FECFE
:1038F0000BF00401380E826F2FEC0BF004012C0E3C
:10390000826F2FEC0BF083EC1AF011EF14F007A884
:10391000FAEF1CF00101800E006F1A0E016F060E07
:10392000026F000E036F4BC104F14CC105F14DC194
:1039300006F14EC107F131EC1FF003BF40EF1DF05F
:103940008CEC1DF04BC100F14CC101F14DC102F1F5
:103950004EC103F107823EEC1EF018C104F119C1FB
:1039600005F11AC106F11BC107F1F80E006FCD0E6B
:10397000016F660E026F030E036F31EC1FF00E0E27
:103980000C6E00C10BF009EC09F00F0E0C6E01C1BA
:103990000BF009EC09F0100E0C6E02C10BF009ECF3
:1039A00009F0110E0C6E03C10BF009EC09F007844D
:1039B00001012CEC20F057C100F158C101F107942E
:1039C0000A0E0C6E00C10BF009EC09F00B0E0C6E28
:1039D00001C10BF009EC09F00C0E0C6E02C10BF0EA
:1039E00009EC09F00D0E0C6E03C10BF009EC09F0A7
:1039F00040EF1DF007AA40EF1DF0078401012CECF9
:103A000020F057C100F158C101F10794060E0C6E69
:103A100000C10BF009EC09F0070E0C6E01C10BF0B0
:103A200009EC09F0080E0C6E02C10BF009EC09F06C
:103A3000090E0C6E03C10BF009EC09F0078462C19A
:103A400000F163C101F164C102F165C103F10794A2
:103A5000120E0C6E00C10BF009EC09F0130E0C6E87
:103A600001C10BF009EC09F0140E0C6E02C10BF051
:103A700009EC09F0150E0C6E03C10BF009EC09F00E
:103A80000798079A0401805181197F0B0DE09EA8C9
:103A9000FED714EE00F081517F0BE126E750812B19
:103AA0000F01AD6E42EF1DF081EF0AF018C100F179
:103AB00019C101F11AC102F11BC103F1000E046F1B
:103AC000000E056F010E066F000E076F62EC1FF00F
:103AD00029A181EF1DF02051D8B481EF1DF018C14C
:103AE00000F119C101F11AC102F11BC103F1000E6D
:103AF000046F000E056F0A0E066F000E076F62EC72
:103B00001FF0120001010451001305510113065169
:103B100002130751031312000101186B196B1A6B82
:103B20001B6B12002AC182F40401300E82272FEC95
:103B30000BF02BC182F40401300E82272FEC0BF026
:103B40002CC182F40401300E82272FEC0BF02DC122
:103B500082F40401300E82272FEC0BF02EC182F488
:103B60000401300E82272FEC0BF02FC182F40401E8
:103B7000300E82272FEC0BF030C182F40401300E9E
:103B800082272FEC0BF031C182F40401300E822722
:103B90002FEC0BF032C182F40401300E82272FEC9F
:103BA0000BF033C182F40401300E82272FEC0BF0AE
:103BB00012002FC182F40401300E82272FEC0BF08B
:103BC00030C182F40401300E82272FEC0BF031C19A
:103BD00082F40401300E82272FEC0BF032C182F404
:103BE0000401300E82272FEC0BF033C182F4040164
:103BF000300E82272FEC0BF01200060E1E6E060E02
:103C00001F6E060E206E1E2E03EF1EF01F2E03EFFA
:103C10001EF0202E03EF1EF08B84020E1E6E020E8D
:103C20001F6E020E206E1E2E13EF1EF01F2E13EFBE
:103C30001EF0202E13EF1EF08B941200FF0E1F6E4D
:103C40001FC020F0030E1E6E8B841E2E24EF1EF06C
:103C5000030E1E6E202E24EF1EF08B941FC020F04A
:103C6000030E1E6E1E2E32EF1EF0030E1E6E203E41
:103C700032EF1EF01F2E20EF1EF012000101005344
:103C800005E1015303E1025301E1002B01EC1FF0B8
:103C90002CEC20F03951006F3A51016F420E046F45
:103CA0004B0E056F000E066F000E076F42EC1FF003
:103CB00000C104F101C105F102C106F103C107F120
:103CC00018C100F119C101F11AC102F11BC103F1C0
:103CD00007B26FEF1EF036EC1FF071EF1EF031EC03
:103CE0001FF000C118F101C119F102C11AF103C19D
:103CF0001BF112002CEC20F059C100F15AC101F166
:103D0000060E20EC09F0E8CF04F1070E20EC09F0D4
:103D1000E8CF05F1080E20EC09F0E8CF06F1090E16
:103D200020EC09F0E8CF07F131EC1FF000C124F1DD
:103D300001C125F102C126F103C127F1290E046F4B
:103D4000000E056F000E066F000E076F42EC1FF0AD
:103D5000EE0E046F430E056F000E066F000E076F28
:103D600036EC1FF024C104F125C105F126C106F18E
:103D700027C107F142EC1FF000C11CF101C11DF188
:103D800002C11EF103C11FF1120E20EC09F0E8CFB1
:103D900004F1130E20EC09F0E8CF05F1140E20EC2D
:103DA00009F0E8CF06F1150E20EC09F0E8CF07F195
:103DB0000D0E006F000E016F000E026F000E036FFC
:103DC00042EC1FF0180E046F000E056F000E066F18
:103DD000000E076F62EC1FF01CC104F11DC105F15C
:103DE0001EC106F11FC107F136EC1FF06A0E046F09
:103DF0002A0E056F000E066F000E076F31EC1FF0E4
:103E00001200BF0EFA6E200E3A6F396BD890003751
:103E1000013702370337D8B012EF1FF03A2F07EF00
:103E20001FF039073A070353D8B412000331070BC8
:103E300080093F6F03390F0B010F396F80EC5FF082
:103E4000406F390580EC5FF0405D405F396B3F3378
:103E5000D8B0392739333FA927EF1FF04051392710
:103E60001200010151EC20F0D8B012000101035101
:103E70000719346F14EC20F0D8900751031934AFB0
:103E8000800F12000101346B38EC20F0D8A04EEC0A
:103E900020F0D8B0120023EC20F02CEC20F01F0E04
:103EA000366F64EC20F00B35D8B014EC20F0D8A0BD
:103EB0000335D8B01200362F51EF1FF034B13BEC70
:103EC00020F012000101346B045105110611071195
:103ED0000008D8A038EC20F0D8A04EEC20F0D8B0E4
:103EE0001200086B096B0A6B0B6B64EC20F01F0E61
:103EF000366F64EC20F007510B5DD8A48CEF1FF0F7
:103F000006510A5DD8A48CEF1FF00551095DD8A4B5
:103F10008CEF1FF00451085DD8A09FEF1FF00451F3
:103F2000085F0551D8A0053D095F0651D8A0063DA0
:103F30000A5F0751D8A0073D0B5FD8900081362F4C
:103F400079EF1FF034B13BEC20F0346B38EC20F00B
:103F5000D89068EC20F007510B5DD8A4BCEF1FF09F
:103F600006510A5DD8A4BCEF1FF00551095DD8A425
:103F7000BCEF1FF00451085DD8A0CBEF1FF0003F4D
:103F8000CBEF1FF0013FCBEF1FF0023FCBEF1FF055
:103F9000032BD8B4120034B13BEC20F01200010125
:103FA000346B38EC20F0D8B012006DEC20F0200E0D
:103FB000366F003701370237033711EE33F00A0E40
:103FC000376FE7360A0EE75CD8B0E76EE552372F59
:103FD000E1EF1FF0362FD9EF1FF034B12981D890CF
:103FE000120001010A0E346F200E366F11EE29F017
:103FF0003451376F0A0ED890E652D8B0E726E73230
:10400000372FFCEF1FF00333023301330033362F19
:10401000F6EF1FF0E750FF0FD8A00335D8B012001D
:1040200029B13BEC20F01200045100270551D8B013
:10403000053D01270651D8B0063D02270751D8B0EB
:10404000073D032712000051086F0151096F02510B
:104050000A6F03510B6F12000101006B016B026BC1
:10406000036B12000101046B056B066B076B1200FA
:104070000335D8A012000351800B001F011F021F3F
:10408000031F003F4BEF20F0013F4BEF20F0023FBA
:104090004BEF20F0032B342B032512000735D8A05B
:1040A00012000751800B041F051F061F071F043F46
:1040B00061EF20F0053F61EF20F0063F61EF20F057
:1040C000072B342B0725120000370137023703373F
:1040D000083709370A370B3712000101296B2A6BA1
:1040E0002B6B2C6B2D6B2E6B2F6B306B316B326B04
:1040F000336B120001012A510F0B2A6F2B510F0B4A
:104100002B6F2C510F0B2C6F2D510F0B2D6F2E5130
:104110000F0B2E6F2F510F0B2F6F30510F0B306F76
:1041200031510F0B316F32510F0B326F33510F0B77
:04413000336F1200D7
:10BF0000E844F926000C160C2B0C3F0C520C640C68
:10BF1000760C860C960CA50CB30CC10CCF0CDC0C6B
:06BF2000E80CF40C000C1B
:00000001FF
